:020000000C28CA
:10000800FE000308F1000408F2000A08F3001F2BA1
:10001800522BA0000A30A100A2012008F900790D96
:10002800790D0139F400740C83120313031C1E2884
:1000380006151F280611790EF400F40C6920031C1C
:100048002728861528288611790EF4006920031CB4
:100058002F28861430288610790E5C20790CF4003D
:10006800F40C6920031C3A2806153B280611790C64
:10007800F4006920031C4228861543288611790C50
:100088000139F400740C83120313031C4D288614E1
:100098004E28861079085C200130A1020030031C2C
:1000A800A203A202210A0319220A031908005028F0
:1000B8000139F400740C83120313031C6528061419
:1000C80066280610061606120800740C0139F50099
:1000D800750C8312031308008312861280300D20DA
:1000E80086162D08F5002C08F400012106300D2095
:1000F8003008F400F501012133080D2032080D20E5
:1001080020300D2046300D204D300D2020300D20A0
:100118002D08F5002C08F40001213608303A031D9B
:1001280097282030B60036080D2035080D203408F1
:100138000D202E300D2033080D2032080D204D30B3
:100148000D2048300D207A300D203630F400F501AE
:100158002C089C3EF6002D080318013EE63EF700E9
:10016800DA217508A7007408A6002608C022BD2059
:100178007C290530F400F5012C082E3EF6002D08E8
:100188000318013E043EF700DA217508AF00740831
:10019800AE000514A5010E3025020318EB282F0820
:1001A800A4002E08A300250ADC280310A40CA30C25
:1001B800FF3E031DD928231CE528831203130515C8
:1001C800E828831203130511A50A8623CF280511F1
:1001D800862305118623051186230511862305111B
:1001E8008623051186230511862305118623051507
:1001F800862305158623051008003030B200B300A9
:10020800B400B500B6002730750210300319740227
:10021800031C1D29B60AF030F4070318F50AD83074
:10022800F5070729B50A1830F4070318F50AFC3052
:10023800F50703307502E83003197402031C2829F6
:100248001629B40A9C303D21003075026430031928
:100258007402031C33292529B30AF6303D210030E6
:1002680075020A3003197402031830297408B2079A
:100278000800F4070318F50AFF30F507080086128E
:1002880077300D20861600300D201F300D201130DC
:100298000D2011300D201F300D2004300D200E30A0
:1002A8000D2015300D20A401A40AA5010530250252
:1002B80003186B29A50AA30108302302031868292B
:1002C800A30A24080D2060290310A40D5A297330AD
:1002D800A400A5010530250203180800A50AF83076
:1002E800A407861224080D2086161F300D206E29BB
:1002F80083169C187C299B01831230089E210318C1
:100308008B179C18852983120310300D83169B00C8
:1003180083122D089E2103188B179C18912903140A
:100328008312300D83169B0083122C089E2103181C
:100338008B17080083169A0003108B1B03148B136A
:100348001C1555309D00AA309D009C141C110800F6
:1003580053308312A6000530A7000130A602031C03
:10036800A703260A0319270A031DB12986120611B5
:10037800861186140610061606127430A60001307F
:10038800A7000130A6020030031CA703A702260A13
:100398000319270A031DC5292B300D2013300D2002
:1003A8000C300D2004300D204321F52AA001A101B5
:1003B800750874040319FF29A201A20AF51BE8298C
:1003C8000310F40DF50DE1290310A00DA10D75081A
:1003D8007702031DF12974087602031CFB297408AF
:1003E800F6027508031CF703F70220140310F50C36
:1003F800F40CA20BE8292108F5002008F4000800F5
:10040800DB228312310803190800310B0C2A55220C
:1004180083123108023A031D122A7A228312310804
:10042800033A031D182A70233108043A031D1D2AB4
:100438006123FF30A8002F30A9000130A802003046
:10044800031CA903A902280A0319290A0319080089
:10045800212A0310300D83169B001C141A088312DE
:10046800AC00AD01AD00AC010314300D83169B0048
:100478001C141A088312AC070318AD0A2A302D027F
:10048800313003192C020318502A19302D02643018
:1004980003192C02031808001030AC002730AD00F7
:1004A8000800FB308312AC070318AD0AFF30AD0714
:1004B80022302D02603003192C0203186E2A1C30DA
:1004C8002D02853003192C02031C6E2A8430AC00DF
:1004D8001C30AD0019302D02643003192C020318AA
:1004E800792A3030AC002A30AD00702805308312EC
:1004F800AC070318AD0A1C302D02853003192C02F5
:10050800031C912A22302D02603003192C02031893
:10051800912A6030AC002230AD002A302D023130F3
:1005280003192C02031C9C2A6430AC001930AD005E
:100538007028F81083120313861BF814781183129D
:100548000313061B7815781DAB2A0130AC2A00303E
:10055800F000F81DB12A0130B22A00307006031DE0
:100568007819BC2AF818BA2A7816BB2A781278148F
:10057800F8117819F8150800A3008612C0300D206C
:100588008616A5015030250203180800A40105307D
:1005980024020318D82AA50AA40A23082506031D3D
:1005A800CB2A24080D20CB2A2D300D20C62A8312F1
:1005B800B101CF308316860083120618E52AB101EF
:1005C800B10A8618E92A0230B1000619ED2A03306B
:1005D800B1008619F12A0430B100C03083168600B4
:1005E8000800B530F600F701861201300D20013001
:1005F800F6020030031CF703F702760A0319770A9C
:10060800031DFB2A861280300D2086160800FF3055
:10061800AA00AB000130AA020030031CAB03AB02F6
:100628002A0A03192B0A031D0E2B4223AC2132235D
:1006380070208B231D2B01300B1C00398B1D0039BA
:1006480000380319282B9D220B1073088A007208A2
:10065800840071088300FE0E7E0E090083169B013C
:100668001C141A088312B0001530300203183F2BEF
:10067800B008031D412BB001B00A2D2A8B01831647
:100688008501C0308600073083129F0085018601EE
:10069800831681138B150B108B170800F801F901CD
:1006A800AC01AD01AE01AF01B001B101B201B301BE
:1006B800B401B501B60183010B2BB00A1530300225
:1006C800031C682BB001B00A2D2270208312B108D8
:1006D80003190800DB226A2BB00B742B1430B0000E
:1006E8002D2270208312B10803190800DB22762B13
:1006F800781C0800781E812B5522781A842B7A22C0
:1007080078107028000085150000851108007C23EA
:02071800042AB1
:02400E00503F21
:104200000100FF0027004C002700A6002700E20065
:104210002800140028006E002800BE002800F000CE
:10422000290022002200560022007E002200A60063
:1042300023008C002600F70027004C002700A60072
:104240002700E2002800140028006E002800BE00AD
:104250002800F000FF00FF00FF00FF00FF00FF004C
:00000001FF
